:020000040800F2
:1000000000080020311F00086D1E0008711E000846
:1000100000000000000000000000000000000000E0
:10002000000000000000000000000000751E000835
:100030000000000000000000791E00087D1E00087E
:10004000B11F0008B11F0008B11F0008B11F000850
:10005000B11F0008B11F0008B11F0008891E000869
:1000600000000000B11F0008B11F0008B11F000808
:10007000B11F0008B11F000800000000C51E0008E5
:100080000000000000000000000000000000000070
:10009000B11F00080000000000000000B11F0008B0
:1000A00000000000B11F0008000000000000000078
:1000B000B11F0008B11F0008000000000000000090
:1000C00010B5064C2378002B07D1054B002B02D02E
:1000D000044800E000BF0123237010BD040000208D
:1000E00000000000FC1F0008044B10B5002B03D0DB
:1000F0000349044800E000BF10BDC04600000000F6
:1001000008000020FC1F0008002243088B4274D323
:1001100003098B425FD3030A8B4244D3030B8B4208
:1001200028D3030C8B420DD3FF22090212BA030C11
:100130008B4202D31212090265D0030B8B4219D3F2
:1001400000E0090AC30B8B4201D3CB03C01A524112
:10015000830B8B4201D38B03C01A5241430B8B425A
:1001600001D34B03C01A5241030B8B4201D30B0343
:10017000C01A5241C30A8B4201D3CB02C01A52416A
:10018000830A8B4201D38B02C01A5241430A8B422D
:1001900001D34B02C01A5241030A8B4201D30B0216
:1001A000C01A5241CDD2C3098B4201D3CB01C01A30
:1001B000524183098B4201D38B01C01A524143093A
:1001C0008B4201D34B01C01A524103098B4201D328
:1001D0000B01C01A5241C3088B4201D3CB00C01A95
:1001E000524183088B4201D38B00C01A524143080D
:1001F0008B4201D34B00C01A5241411A00D2014632
:10020000524110467047FFE701B5002000F006F8A4
:1002100002BDC0460029F7D076E770477047C04658
:10022000002B11D1002A0FD1002900D1002802D0C3
:100230000021C943081C07B4024802A140180290DB
:1002400003BDC046D9FFFFFF03B4684601B502985D
:1002500000F006F8019B9E4602B00CBC7047C046F9
:10026000F0B54F464646D646C0B5040082B00D00F4
:10027000914698468B422FD82CD04146484600F0F4
:10028000B1F829000600200000F0ACF8331A9C46B3
:10029000203B9A4600D576E04B46524693401F00DD
:1002A0004B46624693401E00AF4228D825D05346A5
:1002B000A41BBD41002B00DA7BE00022002300924A
:1002C00001930123524693400193012362469340D8
:1002D000009318E08242D0D90022002300920193BB
:1002E0000A9B002B01D01C605D600098019902B050
:1002F0001CBC90469946A246F0BDA342D7D9002225
:100300000023009201936346002BE9D0FB07984637
:10031000414672080A437B0866460EE0AB4201D1B3
:10032000A2420CD8A41A9D41012024196D4100213C
:10033000013E24184D41002E06D0AB42EED9013EBD
:1003400024196D41002EF8D10098019953460019E7
:100350006941002B23DB2B005246D3402A00644620
:10036000E2401C0053461500002B2DDB26005746AB
:10037000BE40330026006746BE403200801A9941D5
:1003800000900191ACE7624620239B1A4A46DA406E
:100390006146130042468A4017001F4380E76246C9
:1003A00020239B1A2A0066469A402300F3401343F9
:1003B000D4E76246202300219B1A0022009101927B
:1003C0000122DA40019280E72023624626009B1A30
:1003D000DE402F00B0466646B74046463B003343FA
:1003E000C8E7C04610B5002903D100F007F8203057
:1003F00002E0081C00F002F810BDC0461C210123D9
:100400001B04984201D3000C10391B0A984201D3F7
:10041000000A08391B09984201D30009043902A2D5
:10042000105C40187047C04604030202010101013C
:100430000000000000000000FA210A4B10B58900FE
:1004400004001868FFF760FE00F066F8012300283A
:1004500005D100222100013800F028F800231800FF
:1004600010BDC046000000204021084A10B51368A6
:1004700000200B431360FFF7DFFF041E02D00124AE
:10048000200010BD01F098FCFAE7C04600200240B1
:10049000024A1368013313607047C04624000020ED
:1004A000014B18687047C04624000020FF22032338
:1004B00030B51400C5B22B40DB009C4089010A40D6
:1004C000E4439A4000280BDB0C4B80089C46C02379
:1004D000800060449B00C1580C402243C25030BD94
:1004E0000F2307492B408C46083B9B089B00634425
:1004F000D9690C402243DA61F1E7C04600E100E02F
:1005000000ED00E01F2318401E3B8340014A1360AA
:100510007047C04600E100E00A4A431E01209342B2
:100520000ED8C021084A09485360036A09061B0215
:100530001B0A0B4303620023002093600733136000
:100540007047C046FFFFFF0010E000E000ED00E054
:10055000054A1368042803D004218B4313607047B5
:1005600018431060FBE7C04610E000E07047C0464B
:1005700010B5FFF7FBFF10BDF0B5DE4657464E46FF
:100580004546E0B50B6883B09C46002B79D001232B
:100590009A46614B00229846634601910093544667
:1005A0009440009D254068D0019B102759680B009E
:1005B000BB439946022B6BD053009C4603236646EF
:1005C000B34001267642B346D9444E46DB43012E62
:1005D00000D87DE0046867461C40A14603240C4017
:1005E000BC404F463C4367460460C4682340019CBE
:1005F000A468BC402343C36080235B0519423CD000
:1006000056460327454C1740636B33436363444CA2
:10061000BE00A4460F2793089B006344B740B4462E
:10062000A0269C68F605BC43B0420BD03D4EB042BC
:100630006CD03D4EB1460226484500D0062667469E
:10064000BE4034439C604346EC431B68CE035BD4FE
:1006500023404646336073688E0353D42340464696
:100660007360B368CE024BD423404646B360F36850
:10067000890243D423404146CB60009B0132D340E2
:100680008DD103B03CBC90469946A246AB46F0BD26
:10069000D3089B00C3181E6AB146072637001740CF
:1006A000BE000F27B740BB46B4464F465E46B74331
:1006B000019EB94637696646B740BC464F46664616
:1006C00037431F6253009C4603236646B340DB4317
:1006D0008768019E1F40BB46F7686646B740B9462B
:1006E0005F464E4637438760466837005646A74305
:1006F0000C09344094403C4344606BE72B43BAE719
:100700002B43B2E72B43AAE72B43A2E756466746A3
:10071000BE40344396E7C04600040140001002404A
:10072000000001400004005000080050002A01D1E0
:10073000816270478161FCE7044B10B55A69104231
:1007400002D0586101F048F910BDC04600040140D4
:100750000C23244A10B5D1680B40082B2BD00C2B4E
:1007600012D0042B07D08020536800021B045B0FBB
:100770000133984010BD10681B4BC006C0171840CD
:100780001A4B9C466044F5E78B0219481B0FC45C6A
:100790000902D368890F0131DB030ED41368DB062D
:1007A00015D563011B1B9801C01AC0000019000277
:1007B000FFF7AAFCDEE70F48DCE76001001B8301BE
:1007C000181AC00000190002FFF79EFCD2E763016F
:1007D0001B1B9801C01AC00000198002FFF794FC8F
:1007E000C8E7C0460010024000E548FF0024F400BE
:1007F0006C20000800093D00F0B5D6464F4646463D
:10080000C0B5040082B0002800D123E10C25802669
:10081000B94B7602DA681540DA6803681640DA07E1
:1008200033D5082D00D145E10C2D00D13FE18020CA
:1008300061684002814200D146E1A022D202914289
:1008400000D13BE2AC4FAD4B3A681A403A603B688E
:10085000AB4A03400193019B3B6813403B60002976
:1008600000D035E1FFF71CFE80239B0281469846AD
:1008700006E0FFF715FE4B46C01A642800D9A2E136
:1008800042463B681342F4D123689A0700D5ABE097
:10089000DA062AD5002D00D1D4E0A369964E002BAC
:1008A00000D1BCE1802332685B0013433360FFF763
:1008B000F7FD80278046BF0006E0FFF7F1FD4346C5
:1008C000C01A022800D97EE133683B42F5D0736834
:1008D0008C4A1340226A134373607268E369120200
:1008E0001B06120A1343736023681A0719D563693C
:1008F000814E002B00D17DE10122336D134333651E
:10090000FFF7CEFD02230700984605E0FFF7C8FD7C
:10091000C01B022800D956E14246336D1A42F5D079
:1009200023685B0741D580230020734A5B05916BE8
:100930008246194204D1916B0B43936301239A467B
:100940008027714E7F0033683B4200D12BE180222B
:10095000A3685200934200D1BAE1002B00D107E115
:10096000A021C9008B4200D1D1E1634B67491A6DC8
:100970000A401A651A6D66490A401A65FFF790FD2C
:100980008026644B81465C4FB600984606E0FFF730
:1009900087FD4B46C01A404500D914E13B6D3342F8
:1009A000F5D05346012B00D182E1636A002B19D0A8
:1009B0000C2D00D191E1022B00D146E14E4C564A5C
:1009C0002368802513402360FFF76AFDAD0406000D
:1009D00005E0FFF765FD801B022800D9F3E02368DE
:1009E0002B42F6D1002036E02022E3681A4204D0E0
:1009F00041489343016811430160042D33D00C2D0D
:100A00002FD03D4E002B00D1DFE0092132680427B2
:100A10008A4313433360FFF743FD804606E0FFF748
:100A20003FFD4346C01A022800D9CCE033681F427C
:100A3000F5D07268236939491B020A401343736079
:100A4000236825E72C4B1B689B0500D46CE0A36949
:100A5000002B69D1012002B01CBC90469946A246E9
:100A6000F0BD002ECDD1244A1268520701D5002BCB
:100A7000F0D0214E226971682848120201400A43D1
:100A80000921726032688A4313433360FFF760FEC6
:100A9000F368234A1B061B0FD35CD840214B186018
:100AA0000020FFF7C9FC0028D5D12368F0E6002E0E
:100AB00000D1BCE6104A1268920300D4E5E66268F1
:100AC000002A00D0E1E6C5E70B4A13680B43136028
:100AD000FFF7E6FC8027084B81469846BF0205E0F9
:100AE000FFF7DEFC4B46C01A64286CD843461B68EF
:100AF0003B42F5D02368C8E600100240FFFFFEFF2E
:100B0000FFFFFBFFFF1FFFFF00700040FFFEFFFF26
:100B1000FFFBFFFF88130000FFFFFFFEFFE0FFFF6A
:100B200078200008000000207E4A7F485168236A30
:100B30000140194351605068E1690002000A09064A
:100B400001435160D16880225B0B013312029A404D
:100B500013000A067549120F8A5C0020D340744ABC
:100B60001360FFF769FC002800D074E72368BCE637
:100B70006C4E704A336D802713403365336D6E4A77
:100B8000BF0013403365FFF78BFC6C4B81469846E2
:100B900005E0FFF785FC4B46C01A404513D8336D7E
:100BA0003B42F6D1FDE633683B433360FFF778FC08
:100BB000804633683B4200D0C9E6FFF771FC4346EC
:100BC000C01A6428F5D9032045E70122336893430E
:100BD0003360FFF765FC04230700984604E0FFF745
:100BE0005FFCC01B0228EED8424633681A42F6D199
:100BF00023684DE60122336D93433365FFF750FCC4
:100C000002230700984604E0FFF74AFCC01B0228B5
:100C1000D9D84246336D1A42F6D1236881E633684B
:100C2000444A13403360FFF73BFC80239B000700DE
:100C3000984604E0FFF734FCC01B0228C3D84246A4
:100C400033681342F6D123684FE6364D3C4A2B6891
:100C5000802613402B60FFF723FCB604070004E056
:100C6000FFF71EFCC01B0228ADD82B683342F7D11A
:100C7000E16AA36AEA680B4332490A401343226BD4
:100C800080241343EB6080232A685B0413432B60AA
:100C9000FFF706FC234D0600A40404E0FFF700FC68
:100CA000801B02288FD82B682342F7D00020D2E681
:100CB0001C4A2549936B0B40936376E68023194ABF
:100CC000DB0211680B431360136803431360FFE6F4
:100CD000144A116D0B43136550E6124BA16ADA6892
:100CE00080235B02134001208B4200D0B3E6F02347
:100CF000E16A9B0313408B4200D0ACE6C0200004A5
:100D00000240206B101A421E9041C0B2A3E6054B70
:100D10000139186DFF3901431965196D0A431A65C8
:100D20002CE6C04600100240FF1FFFFF782000089D
:100D300000000020FFFEFFFFFFFBFFFF8813000005
:100D4000FFFFFFFEFFFF02FFFFFFFFEFF8B5CE46FC
:100D50004746040080B50D0000280DD001235849F6
:100D60000A681A40AA420CD20A689A432A430A60C7
:100D70000A681340AB4204D001200CBC904699464F
:100D8000F8BD23689A0706D5F0204E49CA68824309
:100D9000A0680243CA60DB0728D54A4A6368126824
:100DA000022B52D0032B53D0012B76D09205E3D5E2
:100DB0000321444EF2688A431343F360FFF770FB4C
:100DC00063680700022B58D0032B69D0012B42D057
:100DD0000C2398463C4B994604E0FFF761FBC01B8F
:100DE000484548D84246F3681A42F6D10121344AB0
:100DF00013680B40AB4205D913688B43136013682B
:100E00001942B9D123685A0706D52E492F48CA6816
:100E10000240E0680243CA601B0707D529492369DD
:100E2000CA682B48DB0002401343CB60FFF790FCFD
:100E3000244B284ADB681B061B0FD35CD840264B8B
:100E400018600020FFF7F8FA97E79203B0D493E711
:100E50009201ADD490E70B3398461B4B994604E0C2
:100E6000FFF71EFBC01B484505D84246F3681340F8
:100E7000042BF5D1BAE703207FE70A339846124BDB
:100E8000994604E0FFF70CFBC01B4845F3D84246E7
:100E9000F3681340082BF5D1A8E7520788D46BE715
:100EA00009339846084B994604E0FFF7F9FAC01B4E
:100EB0004845E0D84246F36813400C2BF5D195E73E
:100EC000002002400010024088130000FFF8FFFFDE
:100ED000FFC7FFFF7820000800000020014B1868C2
:100EE0007047C04600000020044B054ADB685B05E4
:100EF0005B0FD35C034A1068D84070470010024073
:100F00008820000800000020044B054ADB689B0491
:100F10005B0FD35C034A1068D84070470010024052
:100F20008820000800000020F8B5CE464746036838
:100F300080B504009A062ED5802300205C4A5B050C
:100F4000916B8046194204D1916B0B43936301234B
:100F500098468026574D76002B68334244D065680A
:100F6000C020C0212F002A00514E8003336889021F
:100F700007400A4003409F4256D08A424AD0336D10
:100F8000194000D08FE04A490B6D1A4343460A6569
:100F9000012B39D023689A0706D50C204449CA6C26
:100FA0008243A0680243CA645A0706D540494248B2
:100FB000CA6C0240E0680243CA641A0706D53C497D
:100FC0003E48CA6C024020690243CA6400201B06E6
:100FD00006D5374A3A49D36C0B4061690B43D36459
:100FE0000CBC90469946F8BD2B6833432B60FFF745
:100FF00057FA070004E0FFF753FAC01B642850D8E3
:101000002B683342F7D0AAE78B6B2E4A13408B63D1
:101010002368C0E7336801209B03E1D4336D13409C
:1010200036D0934205D130E0336D194028D091423B
:1010300026D023689B0623D580211D4E0903306DE1
:10104000376D214B39433165316D204F03403940B5
:1010500031653365C30513D5FFF722FA80251C4B94
:101060000700AD00994604E0FFF71AFAC01B484597
:1010700017D8336D2B42F7D0C022656892022A4000
:10108000C0239B029A4200D07DE7C027BF032F40B8
:10109000074A104913680B401F431760C022920291
:1010A00071E703209CE7914200D16CE7C1E7C0469D
:1010B0000010024000700040FFF3FFFFFFCFFFFF72
:1010C000FFFFF3FFFFFFFFEFFFFFFCFFFFFFF7FF57
:1010D00088130000FFFFCFFF80220368D2059042F3
:1010E0000ED00C4A90420BD0802293430A691343DE
:1010F00003608B68C3620B6883620123436170479E
:10110000702293434A681343034A1340CA68134347
:10111000EAE7C04600080140FFFCFFFF70B5041E6F
:1011200014D03923C35CDBB2002B0AD0022339254B
:1011300020686355211DFFF7CFFF01230020635571
:1011400070BD3822835400F057FEEFE70120F7E727
:1011500001210368DA680A43DA60072298680240CE
:10116000062A02D01A680A431A6000207047C04657
:1011700001210368DA688A43DA60186A034A104278
:1011800002D11A688A431A600020704711110000CA
:10119000382370B5C25C012A58D001240222C454FD
:1011A0000133C25403684B4D9A682A409A600A681A
:1011B000402A00D174E04BD9602A2ED057D9702A2A
:1011C0001BD08024A401A2420FD19A68424C4D68E2
:1011D00014408A68C9682A4309020A4322439A6074
:1011E00080229968D2010A439A6039230122C254AD
:1011F0000022013BC254002070BD9A68364C4D68F5
:1012000014408A68C9682A4309020A4377212243A5
:101210009A609A680A439A60E7E710251C6A4A6850
:10122000AC43C9681C629D692C4E090335402943B3
:10123000A0251C6A99617021AC43120122431A62F5
:101240009A688A4309390A439A60CEE70220D3E7B5
:10125000102A04D03BD9202A01D0302AC5D17024CD
:101260009968A143693C22430A439A60BDE7502A2A
:10127000BBD14D68CA68196A1E6A1201A6431E6274
:10128000F0269C69B44322430A24A14329439A616E
:10129000196270219A688A4319390A439A60A4E74F
:1012A0004D68CA68196A1E6A1201A6431E62F026BA
:1012B0009C69B44322430A24A14329439A611962D9
:1012C00070219A688A4329390A439A608DE7002A77
:1012D000C5D08AE78800FFFFFF00FFFFFF0FFFFF79
:1012E0007047C0467047C0467047C0467047C0460A
:1012F0000222036810B5196904000A4202D0D968B5
:101300000A4254D1042219690A4202D0D9680A4219
:101310003AD1082219690A4202D0D9680A4225D175
:10132000102219690A4202D0D9680A420ED101225C
:1013300019690A4202D0D9680A424ED1402219697D
:101340000A4202D0D9680A4241D110BD213A1A613D
:1013500019322276DA69C0239B0020001A4243D05A
:10136000FFF7C0FF002323762368E0E7113A1A61F4
:10137000DB690D32227620009B0741D0FFF7B2FFD8
:10138000002323762368CBE7093A1A6107322276D5
:101390009A69C0239B0020001A422ED1FFF7A0FFBC
:1013A0002000FFF7A1FF002323762368B1E7053A69
:1013B0001A619B69043202769B071BD1FFF790FFED
:1013C0002000FFF791FF0023237623689AE7813AF4
:1013D0001A612000FFF78AFFB7E7033A1A6120007D
:1013E00000F0D2FA2368A9E7FFF77AFF2000FFF7A1
:1013F0007BFFB7E7FFF776FFE5E7FFF773FFD2E77D
:10140000FFF76EFF2000FFF76FFFB9E7F0B5382553
:10141000435D012B15D039260223702704688355BC
:101420006268A368BA430F6849683A438027BB43A0
:101430000B436260A36001238355002343550020C2
:10144000F0BD0220FCE7C046F8B504002569A3689A
:1014500002682B436569C1692B4310687A4D0B43C1
:10146000284003431360536878480340E06803430F
:1014700077485360A36982420ED0256A90682B4357
:10148000744D284003439360734B9A4235D001203A
:10149000002323666366F8BD91686E4801400B43E4
:1014A000C021936080226D480901C36CD2000B40BB
:1014B000934278D032D980221201934277D08B4266
:1014C000E5D180231B026268510089189942DED859
:1014D00011039942DBD300275608190E1802801910
:1014E00079410023FEF79CFE5D4BC2185D4B9A428A
:1014F000CDD82368D8600020CAE7584BDA6C0C239B
:101500001340594AD35C80221202914244D0082BE6
:1015100000D993E0554A9B00D3589F46002BB6D183
:10152000FFF7E2FC03000020002BCCD1B0E7FFF76F
:101530000FF963685B0818186168FEF7E5FD03049E
:1015400000201B0C1A004A49103A8A429FD8226890
:10155000D3609DE7FFF7D8FC63685B081818EBE7DA
:101560006368580880231B029C466044E4E7FFF749
:10157000BBFC63685B081818DEE7384B61681B68C2
:101580004808DB061CD43B4B9C466044FEF7BCFD80
:1015900003041B0C0020D5E7082B00D977E7364A57
:1015A0009B00D3589F46FFF7D3F80300BBE7314AAF
:1015B00003689446DB063148DB170340634482E747
:1015C0002F4BE1E7FFF7C4F8636840005B08C018E1
:1015D0006168FEF799FD0004000C0300244A103BEB
:1015E000934200D953E70F2302009A4313000007E8
:1015F0002268400F1843D060002049E7FFF784FCC1
:10160000E2E7164B61681B684808DB0619D51D4BDD
:101610009C466044FEF778FD0004000CDDE7FFF710
:1016200063FCD1E763686168580880235B029C46CD
:101630006044FEF769FD0004000CCEE701200023A2
:1016400080E7114BE4E7C046F369FFEFFFCFFFFFF0
:1016500000480040FFF4FFFF00440040001002403B
:1016600000FDFFFFFFFC0F005C20000814200008B5
:10167000EFFF00000024F4003820000800E548FFD8
:1016800000093D0000127A000048E801436A30B5C5
:10169000DA0706D50168284C4A682240846A22434A
:1016A0004A609A0706D50168244C4A682240C46AF9
:1016B00022434A605A0706D50168214C4A682240F5
:1016C000046B22434A601A0706D501681D4C4A681C
:1016D0002240446B22434A60DA0606D501681A4C60
:1016E0008A682240846B22438A609A0606D5016884
:1016F000164C8A682240C46B22438A605A060AD577
:101700000168134D4A68046C2A4022434A608022D3
:101710005203944209D01B0606D502680D4953684E
:101720000B40816C0B43536030BD4A680A4C224029
:10173000446C22434A60EEE7FFFFFDFFFFFFFEFF20
:10174000FFFFFBFFFF7FFFFFFFEFFFFFFFDFFFFF5D
:10175000FFFFEFFFFFFFF7FFFFFF9FFFF0B5C6465C
:1017600007000C001600984600B5069D3A6801E097
:101770006B1C0AD1D36923401B1B59424B41B34216
:10178000F6D0002004BC9046F0BDFEF789FE43462B
:10179000C01AA84201D8002DE8D13B6808491A6850
:1017A00003200A401A609A68A331FF318A439A6085
:1017B000202300227B67BB675033FA54E2E7C04620
:1017C0005FFEFFFFF0B54746CE4680B51F00436F72
:1017D000040083B00D0016000220202B47D1002901
:1017E0004AD00138002A42D08023A2685B019A4285
:1017F00044D07023E25C012A38D00122E254002355
:10180000E36721336367FEF74BFE50230022E65265
:101810000233E65280239146A26880465B019A42D9
:1018200042D05223E35A002B2ED0522609E02A78C8
:1018300001359A62A35B013B9BB2A353A35B002BD0
:1018400022D000974346002280212000FFF786FF28
:10185000002822D12368002DE9D14A461288D205FA
:10186000D20D9A6202239C46E144E3E7022003B0D2
:101870000CBC90469946F0BD0120F8E72369002B87
:10188000B7D10142B5D0F2E700974346002240218C
:101890002000FFF763FF002801D00320E7E72023A3
:1018A00063675033E054E2E72369002BB9D1A946BE
:1018B0000025B6E7002330B50400C36783B0FEF708
:1018C000EFFD236805001A6812070BD41B685B073D
:1018D00017D42023002200206367A3675033E2540B
:1018E00003B030BD80210D4B00220093890303001B
:1018F0002000FFF733FF00280ED123681B685B0729
:10190000E7D58021054B00220093C9032B0020005E
:10191000FFF724FF0028DCD00320E1E7FFFFFF01F1
:1019200010B5041E27D0436F002B1FD024230121A4
:1019300022686367136820008B431360FFF784FD00
:10194000012818D0636A002B17D123680D495A6803
:1019500020000A402A215A609A688A439A601A68CD
:1019600029390A431A60FFF7A5FF10BD702283547E
:1019700000F05AFADAE70120F7E72000FFF786FEC9
:10198000E3E7C046FFB7FFFF8023026810B5DB0521
:101990009A4200D010BD0F4C032120780130C0B214
:1019A000FEF738FCA023C9B22170DB058022012993
:1019B0000BD0022904D112039A6106229A61E9E749
:1019C00092029A610C229A61E4E7D2029A610A2299
:1019D0009A61DFE720000020A0230100DB051A69DF
:1019E00010B59143784C29D06278002A26D110286E
:1019F0003AD0202828D040285ED0802800D172E03C
:101A00008022520090423FD080229200904200D12A
:101A10008EE08023DB00984200D1B8E080231B01D8
:101A2000984205D11423012268496948FFF7CAFE8C
:101A3000012368486370FFF79BFB04E06548FFF7EC
:101A400087FB0023637010BD5A69920762D55A69FB
:101A500052072AD55B691B07EAD4142301225E4989
:101A60005B48FFF7AFFEE3E75A69920734D55A693E
:101A7000520748D55B691B07DAD414230122574962
:101A80005348FFF79FFED3E75A69920778D55A6902
:101A9000520700D482E05B691B07C9D414230122DA
:101AA0004F494B48FFF78EFEC2E7142301224D49F0
:101AB0004748FFF787FEBBE75A69920731D55A6955
:101AC000520748D55B691B07B2D41423012246494B
:101AD0003F48FFF777FEABE71423012243493C4818
:101AE000FFF770FEA4E75A6992073BD55A6952077F
:101AF0003FD55B691B079BD4142301223C49344822
:101B0000FFF760FE94E7142301223A493048FFF7BB
:101B100059FE8DE71423012237492D48FFF752FE65
:101B200086E71423012235492948FFF74BFE7FE75A
:101B30005A69920739D55B695B073DD5A023DB0560
:101B40005B691B0700D573E7142301222C49204849
:101B5000FFF738FE6CE7142301222A491C48FFF7DF
:101B600031FE65E71423012227491948FFF72AFEB1
:101B70005EE71423012225491548FFF723FE57E7A6
:101B80001423012222491248FFF71CFE50E71423B8
:101B9000012220490E48FFF715FE49E714230122D0
:101BA0001D490B48FFF70EFE42E7142301221B4993
:101BB0000748FFF707FE3BE71423012218490448B2
:101BC000FFF700FE34E7C04620000020DC200008BC
:101BD0006400002028000020A420000898200008AD
:101BE000C8200008A0200008B020000890200008AD
:101BF000BC200008942000089C200008A8200008B1
:101C0000D4200008AC200008B4200008B820000848
:101C1000C0200008D8200008C4200008CC200008FC
:101C2000D02000082049214A0B6830B51A40802393
:101C30001B0113430B60012399B00B93A023DB021C
:101C40000C9380235B021593A0235B0316938023E0
:101C50000225DB030BA817931495FEF7CDFD0F2388
:101C600000240121009368460C3B019302940394E5
:101C70000494FFF76BF805A805950794FFF754F94E
:101C8000FFF72CF9FA218900FEF73EFAFEF744FC33
:101C90000420FEF75DFC0120002200214042FEF7F7
:101CA00005FC19B030BDC04600700040FFE7FFFFE3
:101CB000F0B501248BB0FEF7D7FBFFF7B3FF374B2E
:101CC000A026DA6AF6052243DA62DA6A3000224098
:101CD0000192019A0222D96A0E271143D962DB6A66
:101CE0000E211A4002920122029BFEF71FFD0323E0
:101CF0000694002405A93000089305970794FEF781
:101D00003BFCFC239B000593254B05A93000069363
:101D10000794FEF731FCC0231B010593214B05A955
:101D2000300006930794FEF727FC002200210720CD
:101D3000FEF7BCFB0720FEF7E5FB1B481B4B84604E
:101D4000036096239B0143600823C46043610461E0
:101D50008461C46104624462FFF7E2FD8023144D94
:101D6000DB052B60134B2800EB606C60AC602C61D2
:101D7000FFF7D4F9802305A95B0128000593FFF73D
:101D800007FA202303A9280003930494FFF73EFBDE
:101D9000B7612800FFF7DCF9FEE7C04600100240FB
:101DA00000003110000021106400002000440040B9
:101DB000280000207F3E000001210E4B10B55A6B19
:101DC00005200A435A638022996B52050A439A639D
:101DD000002100224042FEF769FB02200022002180
:101DE0004042FEF763FB0120002200214042FEF743
:101DF0005DFB10BD001002408023026810B5DB05BA
:101E00009A4200D010BD0121064A0F20936B0B436C
:101E1000936300210022FEF749FB0F20FEF772FBBF
:101E2000F0E7C0460010024000B50D4B026887B0D5
:101E30009A4201D007B000BD80230A4A9B02916BF1
:101E400009480B439363C0230193BE3B02930322D3
:101E5000002301A9039304920593FEF78DFBE9E7A4
:101E60000044004000100240000400507047C0468B
:101E7000FEE7C0467047C0467047C04610B5FEF743
:101E800007FBFEF775FB10BD10B51020FEF754FCE4
:101E90002020FEF751FC4020FEF74EFC8020FEF78C
:101EA0004BFC80204000FEF747FC80208000FEF7BE
:101EB00043FC8020C000FEF73FFC80200001FEF7BD
:101EC0003BFC10BD10B50248FFF712FA10BDC0462A
:101ED000280000208022104B520019680A431A6023
:101EE000DA680E490A40DA601A680D490A40012191
:101EF0001A609A688A439A601A680A490A401A6006
:101F0000DA6809490A40DA6000221A618022074B28
:101F100012059A607047C046001002400C40FF88CE
:101F2000F6FFF6FEFFFFFBFFFFFF02FF00ED00E004
:101F30001348854613480168090E134A914205D19A
:101F4000124813490160134813490160002103E05E
:101F5000124B5B58435004311148124B42189A42BD
:101F6000F6D3114A02E00023136004320F4B9A4269
:101F7000F9D3FFF7AFFF00F01DF8FFF799FEFEE77A
:101F800000080020040000001F0000003410024080
:101F9000010000000000014000000000F0200008E7
:101FA000000000200400002004000020E4000020C5
:101FB000FEE7000070B500260C4D0D4C641BA4100C
:101FC000A64209D1002600F019F80A4D0A4C641BFC
:101FD000A410A64205D170BDB300EB589847013656
:101FE000EEE7B300EB5898470136F2E7E820000827
:101FF000E8200008E8200008EC200008F8B5C046FA
:10200000F8BC08BC9E467047F8B5C046F8BC08BC92
:042010009E46704731
:102014006E150008541500087A1500083C160008CF
:102024002E1500083C1600083C1600083C16000853
:10203400601500081E160008FC15000802160008AA
:102044008E140008C41500088E1400088E140008AD
:102054008E1400082416000800101010041010102C
:102064000210101008000000030406080C101820C9
:102074003000000000000000000000000102030422
:102084000607080900000000010203042A000000FA
:102094003000000023000000310000003200000086
:1020A400330000003400000035000000360000005A
:1020B4003700000038000000390000004C00000028
:1020C40044000000520000004100000055000000E0
:0C20D4004200000058000000590000000D
:0820E00080E1FF7F0100000018
:0420E800E900000803
:0420EC00C100000827
:0420F00000002000CC
:0400000508001F319F
:00000001FF
